:0200000048288E
:08000800831204288200523427
:100010004534503420343D34203400345334593482
:10002000533420343D3420340034433420343D34C0
:100030002034003444344F344E3420343D340034C2
:10004000203420344434453443344F34443445342C
:10005000553452342034523443343534003420344F
:10006000203420342034203443344F344434413459
:10007000473445340034203420342034203449348B
:100080004E34563441344C344934443445340034CD
:1000900083018B018A01850186018316F830850072
:1000A00000308600D13081008312AF200030E32081
:1000B0002030A5206428D1200030E3202F30A52057
:1000C0004030E3203B30A52085196428933081001F
:1000D0000B110310322103186428632103185B28D5
:1000E000D1200030E3200730A52010089500122110
:1000F0001508F6200830E3200E30A52011089500E1
:1001000012211608F6201508F6204030E32015309D
:10011000A5201208950012211708F6201608F620CF
:100120001508F6204830E3201A30A520231CA0280B
:100130001308950012211608F6201508F6206428E9
:100140002030F6202030F620642894001408062081
:10015000003A0319AE28F620940AA6280800850163
:100160001E300D213830FF200030DB20D12004303C
:10017000DB200230D7200800051505110800831682
:10018000FF30860083120510851405150608051139
:100190008039031DBF288510831600308600831226
:1001A00008000130FF2008000230FF20080003395A
:1001B0000438FF20080007390838FF2008003F39BD
:1001C0004038FF2008008038FF2008008316FF30E9
:1001D00086008312051085140515060805117F3960
:1001E0008510831600308600831208008C00BF2023
:1001F0008510051405150C088600051108008C00F3
:10020000BF208510051005150C0886000511080093
:10021000A5308E008E0B0A2908008F0008218F0B55
:100220000E29080030309600970064301502031C38
:100230001C299500970A15290A301502031C232949
:100240009500960A1C293030950730301706031D9B
:1002500031292030970030301606031D3129203017
:10026000960008001B3084008001840A21300406B7
:10027000031D3429980199011B3084000B1D3E2970
:100280005F218519D2290B1D43295F21980A2B3044
:10029000180603195329031485190310800D990AB0
:1002A00099195C2143290310800D800D800D800D6C
:1002B000800D800D03100800840A990108000B11BD
:1002C0002530810008001B3084009A019901A301A8
:1002D000A1019001910192019301800D9A0D800D71
:1002E0009A0D990AC5212219D229A20CA10D9A01B1
:1002F000800D9A0D800D9A0D990AC5212219D229D7
:10030000A20C900D05308D009A01800D9A0D800D84
:100310009A0D990A19195C21C5212219D229A20C1A
:10032000910D8D0B8429C0301C05031D9D295C2176
:10033000800D800D990A0130A30006308D009A01CE
:10034000800D9A0D800D9A0D990A19195C21C5210D
:1003500022190000A20C920D8D0B9F29211C12174F
:100360002318B329080006308D009A01800D9A0DDC
:10037000800D9A0D990A19195C21C52122190000D6
:10038000A20C930D8D0BB5290800A20101301A06AD
:100390000319D02902301A060319D12922150800A1
:0803A0002214080003140800F8
:02400E00F13F80
:00000001FF
